:100000000C94D5050C941D060C941D060C941D062D
:100010000C941D060C941D060C941D060C941D06D4
:100020000C941D060C941D060C941D060C9487253B
:100030000C941D060C945E250C941D060C941D0654
:100040000C941D060C941D060C941D060C9438256A
:100050000C941D060C941D060C941D060C941D0694
:100060000C941D060C941D060C941D060C941D0684
:100070000C941D060631FF0974A1010975150026AF
:10008000FF009520750881020976150026FF00956E
:100090002075089102C005010902A1010901A10012
:1000A0008501050919012908150025019508750123
:1000B00081020501093009311581257F95027508F6
:1000C000810609381581257F950175088106050C83
:1000D0000A38021581257F950175088106C0C00583
:1000E000010980A10185021601002637001A81004E
:1000F0002AB700751095018100C0050C0901A10106
:100100008503160100269C021A01002A9C02751024
:1001100095018100C005010906A101050719E02923
:10012000E715002501950875018102950175088183
:1001300001050819012905950575019102950175BB
:100140000391010507190029FF150026FF009506F8
:1001500075088100C00A0025583A253032582025FC
:10016000583A253032580A002D2D2D2D2D2D2D2DAC
:100170002D0A00413A482020613A680A000A546179
:10018000626C653A0A000A002425582052333A2549
:100190003034580A000A5363616E3A0A004B3A241D
:1001A00025583A253032583A2530345820005B2003
:1001B000423A2530325820583A25642825642920AF
:1001C000593A25642825642920563A2564205D0A79
:1001D000005D20002530325820004D3A2425583A41
:1001E000253032583A5B20006D3A556E6B6E6F7752
:1001F0006E3A20253032580A006D3A2425583A25A7
:1002000030345820004B3A2425583A4C61796F75A8
:10021000743A2025730A004B3A2425583A536574E2
:1002200075702E2052333A253034580A004B3A2448
:1002300025583A4E6F7420666F756E640A004D3A09
:100240002425583A4B656E73696E67746F6E0A00A9
:100250004D3A2425583A457874656E6465640A0001
:100260004D3A2425583A4C6F6769746563682D458B
:100270007874656E6465640A004D3A2425583A4CDA
:100280006F6769746563680A004D3A2425583A4DD2
:100290006163616C6C792D3262746E0A004D3A2490
:1002A00025583A4B656E73696E67746F6E2045789A
:1002B000740A004D3A2425583A4558543A205B2593
:1002C0003032582025303258202530325820253001
:1002D00032582025303258202530325820253032EF
:1002E0005820253032585D206370693D25642062B6
:1002F000746E3D2564206C656E3D25640A004D3AA0
:100300002425583A436C617373696332203230306C
:100310006370690A004D3A2425583A436C6173733F
:10032000696331203130306370690A004D3A242509
:10033000583A53657475702E2052333A253034582C
:100340000A004D3A2425583A4E6F7420666F756E38
:10035000640A00413A2425583A4170706C69616E14
:100360006365284D65646961206B657973290A00AE
:10037000523A2425583A4D6F766520746F20242513
:10038000582E2052333A253034580A00523A242548
:10039000583A4661696C20746F206D6F76650A006B
:1003A000523A2425583A4E6F206672656520616482
:1003B00064726573730A00523A2425583A466F7581
:1003C0006E642E2052333A253034580A005D0A00FC
:1003D000253032582000553A2425583A25303258D5
:1003E0003A5B200073005300520025583A253038FC
:1003F0006225730A000A2020303132333435363713
:100400000A004C45443A20253032580A000A4C6F05
:100410006F702073746172742E0A000A5553422063
:10042000636F6E666967757265642E0A000A544DC3
:100430004B3A6563663532392F4C5546413A64363E
:10044000613764660A0009025400030100A0320902
:1004500004000001030101000921110100012240F3
:10046000000705810308000A0904010001030102D5
:1004700000092111010001227F0007058203080005
:10048000010904020001030000000921110100011B
:100490002222000705830320000112011001000041
:1004A0000008EDFEDB0A0101010200012E034100FC
:1004B0004400420020006B006500790062006F007C
:1004C000610072006400200063006F006E0076001F
:1004D0006500720074006500720000000E03740075
:1004E0002E006D002E006B002E0000000403090496
:1004F00073797374656D3A20253034580A00636F40
:100500006E73756D65723A20253034580A003F00CD
:100510004D3E2000433E20000A00257500363A205B
:10052000776865656C5F74696D655F746F5F6D6139
:10053000783A20000A00257500353A20776865650D
:100540006C5F6D61785F73706565643A20000A00C6
:10055000257500343A2074696D655F746F5F6D6155
:10056000783A20000A00257500333A206D61785FE3
:1005700073706565643A20000A00257500323A20E0
:10058000696E74657276616C286D73293A20000A71
:1005900000257500313A2064656C6179282A313074
:1005A0006D73293A20000A092D2056616C75657318
:1005B000202D0A004D3E004D25643E20003F007373
:1005C00065742064656661756C740A00433E2000A2
:1005D0000A002530325820006B6579626F617264C1
:1005E0003A2000041607090B0A1D1B06196405149E
:1005F0001A08151C171E1F202123222E26242D2504
:10060000273012182F0C13280F0D340E33313638C3
:100610001110372B2C352A5829787B79397A504F8D
:10062000515280806368568066805302010355589A
:10063000805780805462595A5B5C5D5E5F80606168
:100640007475673E3F403C414277447646004780A0
:100650004365453248494A4B4C3D4D3B4E3A7D7EC1
:100660007C7F73290A002575002F002575005D2801
:10067000002564002000256400200025640020007F
:100680002564007C0025303258006D6F7573656BF2
:100690006579205B62746E7C782079207620685DB5
:1006A000287265702F61636C293A205B000A092D5E
:1006B000204D61676963202D0A643A09646562759B
:1006C000670A783A096465627567206D61747269BA
:1006D000780A6B3A096465627567206B6579626FA9
:1006E0006172640A6D3A096465627567206D6F75A1
:1006F00073650A763A0976657273696F6E0A733AA2
:10070000097374617475730A633A09636F6E736F6A
:100710006C65206D6F64650A302D343A096C61791F
:100720006572302D34284631302D4634290A506107
:1007300075733A09626F6F746C6F616465720A0059
:100740000A092D20436F6E736F6C65202D0A455387
:10075000432F713A09717569740A6D3A096D6F75A5
:1007600073656B65790A003F0074696D65725F722D
:10077000656164333228293A202530346C580A00E8
:100780006B6579626F6172645F69646C653A20259C
:10079000580A006B6579626F6172645F70726F7482
:1007A0006F636F6C3A2025580A00686F73745F6B33
:1007B0006579626F6172645F6C65647328293A20A1
:1007C00025580A000A092D20537461747573202D71
:1007D0000A004743433A20372E332E3020415652E9
:1007E0002D4C4942433A20322E302E302041565271
:1007F0005F415243483A2061767233350A004F50C8
:1008000054494F4E533A204C554641204D4F555375
:10081000454B45592045585452414B455920434F6B
:100820004E534F4C4520434F4D4D414E44204B4578
:10083000594D41505F53454354494F4E2034303950
:10084000360A004255494C443A20656366353239D0
:10085000202830313A33373A3537204D6172203114
:10086000322032303233290A005649443A20307857
:100870004645454428742E6D2E6B2E292050494440
:100880003A2030783041444228414442206B657917
:10089000626F61726420636F6E766572746572292F
:1008A000205645523A203078303130310A004445E4
:1008B00053433A20636F6E76657274204144422040
:1008C0006B6579626F61726420746F205553420AC0
:1008D000000A092D2056657273696F6E202D0A007B
:1008E0000A6D6F7573653A206F66660A000A6D6F50
:1008F0007573653A206F6E0A000A6B6579626F61E5
:1009000072643A206F66660A000A6B6579626F61ED
:1009100072643A206F6E0A000A6D61747269783AE7
:10092000206F66660A000A6D61747269783A206FFA
:100930006E0A000A64656275673A206F6E0A000AE3
:1009400064656275673A206F66660A000A0A626F1C
:100950006F746C6F616465722E2E2E2000433E20F2
:10096000006D6B5F776865656C5F74696D655F745A
:100970006F5F6D6178203D2025640A006D6B5F77A5
:100980006865656C5F6D61785F7370656564203D57
:100990002025640A006D6B5F74696D655F746F5F1D
:1009A0006D6178203D2025640A006D6B5F6D617874
:1009B0005F7370656564203D2025640A006D6B5F80
:1009C000696E74657276616C203D2025640A006D45
:1009D0006B5F64656C6179203D2025640A006D6B56
:1009E0005F776865656C5F74696D655F746F5F6D77
:1009F0006178203D2025640A006D6B5F776865652E
:100A00006C5F6D61785F7370656564203D2025645F
:100A10000A006D6B5F74696D655F746F5F6D6178FF
:100A2000203D2025640A006D6B5F6D61785F7370F7
:100A3000656564203D2025640A006D6B5F696E74F6
:100A4000657276616C203D2025640A006D6B5F64E1
:100A5000656C6179203D2025640A007768657265C0
:100A60002064656C74613A20637572736F723D2502
:100A7000642C20776865656C3D25640A53656520A4
:100A8000687474703A2F2F656E2E77696B69706584
:100A90006469612E6F72672F77696B692F4D6F756F
:100AA00073655F6B6579730A000A092D204D6F75B8
:100AB00073656B6579202D0A4553432F713A09718F
:100AC0007569740A313A0964656C6179282A313094
:100AD0006D73290A323A09696E74657276616C2801
:100AE0006D73290A333A096D61785F7370656564C7
:100AF0000A343A0974696D655F746F5F6D61780AD5
:100B0000353A09776865656C5F6D61785F7370650C
:100B100065640A363A09776865656C5F74696D6566
:100B20005F746F5F6D61780A0A703A097072696E5E
:100B3000742076616C7565730A643A097365742074
:100B400064656661756C74730A75703A092B310AB5
:100B5000646F776E3A092D310A706775703A092B08
:100B600031300A7067646F776E3A092D31300A0AA6
:100B70007370656564203D2064656C7461202A2073
:100B80006D61785F7370656564202A2028726570D6
:100B9000656174202F2074696D655F746F5F6D618E
:100BA00078290A004C25640A000011241FBECFEFEB
:100BB000D4E0DEBFCDBF04B603FE28C08091B103F0
:100BC0009091B203A091B303B091B4038730904BDE
:100BD000A740B04BD9F41092B1031092B203109217
:100BE000B3031092B40314BE0FB6F894A895809185
:100BF0006000886180936000109260000FBE1092C8
:100C0000010810920008E0E0F8E3099511E0A0E087
:100C1000B1E0EAE4F5E502C005900D92A235B10716
:100C2000D9F723E0A2E5B1E001C01D92A13BB207D4
:100C3000E1F70E9438260C94A32A0C940000FF933D
:100C4000EF93E0915201F0915301309709F009952B
:100C5000EF91FF910895FC018591803011F0EFDF55
:100C6000FBCF0895FF27E0E230E247FF0CC041953B
:100C700097FF09C0EDE26095709580959095611D94
:100C8000711D811D911D27FF02C0219530E350E2A7
:100C9000AA27660F771F881F991FAA1FA41710F095
:100CA000A41B63955A95A9F7AA3008F0A95FA05D27
:100CB000AF93F395611571058105910541F7ED320B
:100CC00011F4EF93F395F21718F43F93F395FBCFDC
:100CD0008F91B5DFFA95E1F70895E991F991859142
:100CE000803021F0853219F0AADFF9CF089520E095
:100CF000E89455915532C1F3503311F468945591ED
:100D00005A3348F4505390F3220F022E220F220F31
:100D1000200D250FF4CF0EF421958991999153362A
:100D200019F3533729F1533559F1BC018827992715
:100D3000E8945C3621F489919991689455915436E0
:100D400039F446EF7EF077FF0DC08FEF9FEF0AC0BA
:100D500055374AE039F0583540E121F0523642E04B
:100D600009F00895FF93EF937DDFEF91FF91B7CFE7
:100D7000FF93EF93FC0181918030B9F360DFFBCFEB
:100D8000FF93EF9368DFF1CFDF93CF93CDB7DEB75B
:100D90002596A3DFCF91DF91089580919D0380FF79
:100DA0000CC06091160170E0759567957595679513
:100DB0006115710559F1862F089581FF06C0609174
:100DC000160170E075956795F3CF6091160170E09C
:100DD00082FD0CC060919E036623A9F0209115014D
:100DE0008091160190E0621730F0BC016038710507
:100DF000F8F28FE7089570E00E94642A622F70E095
:100E00000E94752AF3CF61E070E0D5CF81E00895AC
:100E100080919D0380FF11C08091180190E065E0F2
:100E200070E00E94642A95958795959587958038FE
:100E30009105B0F50097B1F1089581FF0AC0809146
:100E4000180190E065E070E00E94642A959587950E
:100E5000EECF82FF08C08091180190E065E070E05D
:100E60000E94642AE4CF30919E033323B1F0209195
:100E700017018091180190E065E070E00E94642AFB
:100E8000BC013217A0F6832F90E00E94642A622FE3
:100E900070E00E94752ACB01CACF85E090E00895EA
:100EA0008FE7089581E00895E72FF0E093E0EE0FDB
:100EB000FF1F9A95E1F7E60FF11DED51FA4F64918E
:100EC000E62FE295E77090E023E0880F991F2A95BE
:100ED000E1F78E0F911D34E0880F991F3A95E1F7E5
:100EE000E62FEF70E80FF92FF11DEE0FFF1FE05016
:100EF000F8498591949108952FB7F8948091A603AD
:100F00009091A703A091A803B091A9032FBF0895C2
:100F1000E4E5F2E09281891301C01282319692E0F9
:100F2000EA35F907B9F70895A6E5B2E0EFEF90E0EA
:100F30002D91821751F0EF3F19F4211101C0E92FD3
:100F40009F5F9630A9F7EF3F09F408950E2E000C2D
:100F5000FF0BEC5AFD4F828308954F925F926F9280
:100F60007F929F92AF92BF92CF92DF92EF92FF92C9
:100F70000F931F93CF93DF9300D000D01F92CDB774
:100F8000DEB76B837C838D837A018C819D81892B75
:100F900049F08FEFF81204C081E09FEF491719F074
:100FA00080E001C081E080FD6AC00F2D10E0CE2CF2
:100FB000D12C8B81882309F456C0409013035090A4
:100FC000140360901503709016038091AD03909107
:100FD000AE03A091AF03B091B003482A592A6A2A00
:100FE0007B2A2FE1A22EB12C9A2CD301C2010A2C0C
:100FF00004C0B695A795979587950A94D2F780FD7A
:101000002BC081E0A81AB10878F7912CF80193E081
:10101000EE0FFF1F9A95E1F7E95EFC4FEC0DFD1D09
:101020009082E982FA8269817A81892D0F900F90EE
:101030000F900F900F90DF91CF911F910F91FF9024
:10104000EF90DF90CF90BF90AF909F907F906F9088
:101050005F904F900C945407B7018A2D0E9454075B
:10106000019779F2D3CFF80183E0EE0FFF1F8A9545
:10107000E1F7E95EFC4FEC0DFD1D9080D2CF90E0D2
:1010800080E00F900F900F900F900F90DF91CF9115
:101090001F910F91FF90EF90DF90CF90BF90AF9096
:1010A0009F907F906F905F904F90089541E050E047
:1010B00060E070E004C0440F551F661F771F8A95DB
:1010C000D2F740955095609570958091130390915B
:1010D0001403A0911503B091160384239523A6232E
:1010E000B7238093130390931403A0931503B09335
:1010F0001603089541E050E060E070E004C0440F42
:10110000551F661F771F8A95D2F780911303909120
:101110001403A0911503B0911603842B952BA62BD5
:10112000B72B8093130390931403A0931503B093EC
:1011300016030895809112039091E102981301C063
:1011400008958F5F8770FACF1F93CF93DF9300D0FE
:1011500000D01F92CDB7DEB7942F4983252F5A8335
:101160006B837C838D834C815D8181E0452B31F0E5
:101170002F3F19F481E09F3F09F080E0182F117094
:1011800080FD2CC049815A816B817C818D810E94B8
:10119000AD07292F22952F702C3078F42A30A8F42F
:1011A00022502230C8F0812F0F900F900F900F9097
:1011B0000F90DF91CF911F9108952C3011F02F30B7
:1011C00091F793FB112710F9EECF803C28F0803E79
:1011D00050F3815F833038F311E0E5CF10E0E3CFC7
:1011E0001F93CF93DF93E0919703F091980330978B
:1011F00081F0EC0118818091A103812B888390916B
:10120000C102892B88830480F581E02DCE010995E8
:101210001883DF91CF911F910895E0919703F0918A
:101220009803309721F00190F081E02D099480E03F
:1012300008951092E2001092E100E0EEF0E080816B
:1012400081608083E8EDF0E080818F77808319BC36
:10125000E3E6F0E08081816080831092AA02089525
:101260000E941909F89487E797E790930108809303
:10127000000887E090EBDC018093B1039093B20308
:10128000A093B303B093B40388E19CE00FB6F89445
:10129000A895809360000FBE90936000FFCFFC0183
:1012A0008091BE029091BF0286179707A0F061154A
:1012B000710529F49091E8009E779093E80090E002
:1012C0006115710551F4911108C08091E80082FF09
:1012D00032C080E00895BC01F2CF8091C002882323
:1012E000B1F18530B1F18091E80083FD2EC080918D
:1012F000E80082FDEACF8091E80080FFE1CF2091F5
:10130000F20030E06115710519F02830310558F010
:1013100091E02830310509F090E02091E8002E7727
:101320002093E800CDCF81918093F1006150710945
:101330002F5F3F4FE7CF8091C002882341F0853077
:1013400041F08091E80083FFC0CF81E0089582E002
:10135000089583E008952091E4003091E50085E64A
:101360009091EC0090FF06C09091E80090FF06C0BD
:1013700080E008959091E80092FDFACF9091C0022C
:10138000992391F0953091F09091EB0095FD10C06C
:101390004091E4005091E5002417350709F381508E
:1013A0009A01F1F684E0089582E0089583E00895BB
:1013B00081E008958091B80287FF13C08091E80012
:1013C00082FF06C08091E8008B778093E80004C01C
:1013D0008091C0028111F2CF08958091C0028823CC
:1013E000D9F38091E80080FFF8CF8091E8008E77F4
:1013F000ECCF982F9093E900242F762F50E0891797
:1014000031F07091EC002091ED005091F00021FD41
:1014100007C09F5F953071F78093E90081E00895E0
:101420003091EB003E7F3093EB003091ED003D7F3B
:101430003093ED003091EB0031603093EB0070930E
:10144000EC002093ED005093F0002091EE0027FD7A
:10145000E0CF80E008950F931F93CF93DF93CDB734
:10146000DEB7AA970FB6F894DEBF0FBECDBF80914E
:10147000C002882309F44EC11091E9001F708091C9
:10148000EC0080FF39C080E8182B1092E9008091B1
:10149000E80083FF3CC1E8EBF2E080EC92E02091B1
:1014A000F10021938E179F07D1F78091B902833005
:1014B00009F470C018F5813009F447C0823009F48E
:1014C000DAC08091E80083FF14C18091B802909146
:1014D000B9029A3008F00DC1E92FF0E0EE58F54F4F
:1014E0000C94892A4C0B720B790B720B790BD40B71
:1014F000F60B790BF10CFE0C80E0C6CF8A3009F4B4
:10150000A9C08B3009F47DC08930D9F68091B8022A
:101510008132B9F68091BC029091BD02892B89F687
:101520008091E800877F8093E8008091E80082FF47
:101530002CC08091F1008093AC028091E8008B7701
:101540008093E8000E94DA09BCCF8091B802813A0A
:1015500009F0B7CF8091E800877F8093E800809101
:10156000BC029091BD02892B61F060E090E080E0C8
:1015700070E00E944F098091E8008B778093E8002B
:10158000A0CF68E08DEA92E0F3CF8091C002811194
:10159000CCCF97CF8091B802813A09F092CF809159
:1015A000BC029091BD02892BA1F48091E800877F55
:1015B0008093E8008091E80080FFFCCF80911401C7
:1015C0008093F1008091E8008E778093E8000E947C
:1015D000DA098091BC029091BD02019709F071CFA8
:1015E0008091E800877F8093E8008091E80080FF89
:1015F000FCCF809113018093F1008091E8008E77F9
:101600009FCF8091B802813209F05BCF8091BC02FC
:101610009091BD02892B59F48091E800877F8093D7
:10162000E8000E94DA098091BA0280931401809147
:10163000BC029091BD02019709F043CF8091E80070
:10164000877F8093E8000E94DA098091BA02809334
:10165000130137CF8091B802813209F032CF8091E7
:10166000E800877F8093E8000E94DA098091BB023E
:101670008093AA0326CF8091B802813A09F021CF46
:101680008091E800877F8093E8008091E80080FFE8
:10169000FCCF8091AA03AFCF803889F0823849F51A
:1016A0008091BC028F70853020F58093E900809195
:1016B000EB0085FB882780F91092E90006C0809135
:1016C000B5029091B602911182609091E800977FE7
:1016D0009093E8008093F1001092F1008091E8006F
:1016E0008E7731C0282F2D7F21F48823F1F08230AE
:1016F00079F18091E80083FF0AC08091E800877F3C
:101700008093E8008091EB0080628093EB001F7073
:101710001093E900AA960FB6F894DEBF0FBECDBFB6
:10172000DF91CF911F910F9108958091BA0281307E
:1017300001F7933009F080E08093B6021092E9003F
:101740008091E800877F8093E8000E94DA09D1CF7A
:101750008091BA028111F2CF8091BC028F702FEF7D
:10176000280F243030F68093E9002091EB0020FF11
:10177000E5CF933031F48091EB0080628093EB00F1
:10178000DDCF9091EB0090619093EB0021E030E091
:1017900001C0220F8A95EAF72093EA001092EA002E
:1017A0008091EB008860EACF8111A3CF0091BA024B
:1017B0000F778091E3008078802B8093E300809105
:1017C000E800877F8093E8000E94DA098091E800B2
:1017D00080FFFCCF8091E30080688093E30083E08A
:1017E000011101C082E08093C00283CF8058823013
:1017F00008F07FCF2091BA023091BB022C3D83E0EC
:101800003807A1F583E08A838AE289834FB7F89489
:10181000DE01139620E03EE051E2E32FF0E050932A
:101820005700E49120FF03C0E295EF703F5FEF7037
:101830008E2F90E0EA30C0F0C7968D939D932F5F76
:10184000243159F74FBF8091E800877F8093E800EB
:101850006AE270E0CE0101960E944F098091E80093
:101860008B778093E80045CFC096E7CF8091BC028C
:101870009091BD02432F55274330510509F44FC0C5
:1018800078F54130510509F445C084E590E0E6E47F
:10189000F4E04230510509F02CCF2091E800277F79
:1018A0002093E8002091BE023091BF028217930777
:1018B00008F49C0140E02115310509F063C0411195
:1018C00061C08091E80082FDC9CF8091C002882369
:1018D00029F2853019F28091E80083FFF2CFBECF64
:1018E0004132510509F43FC04232510509F001CFA0
:1018F0008330910508F0FDCEFC01EE0FFF1FE55C83
:10190000FE4F0190F081E02D885C9E4FDC018C91B0
:1019100090E01DC082E190E0EAE9F4E0BECF332719
:1019200021303105C1F060F02230310509F0E1CEFF
:10193000ECEAF4E0E4918E2F90E0ECEAF4E007C0EA
:10194000ECEEF4E0E4918E2F90E0ECEEF4E0009702
:1019500009F4CFCEA2CFECEDF4E0E4918E2F90E02D
:10196000ECEDF4E0F4CF8330910508F0C2CE880F9F
:10197000991FFC01EF5BFE4F0190F081E02D89E0A3
:1019800090E08BCF8091C002882309F467CF853027
:1019900009F464CF8091E80083FD60CF8091E80076
:1019A00082FD8FCF8091E80080FF85CF8091F2008B
:1019B00090E02115310519F08830910550F041E093
:1019C000089709F040E08091E8008E778093E80066
:1019D00072CF44914093F100319621503109019624
:1019E000E8CF803809F085CE8091E800877F80932A
:1019F000E8008091B7028093F10070CE811179CE1A
:101A00000091BA02023008F074CE8091E800877F1E
:101A10008093E8000093B7020E94DA09002399F04E
:101A200084E08093C00242E061EC81E00E94F90909
:101A300042E061EC82E00E94F90946E261EC83E059
:101A40000E94F90956CE8091E30087FDE9CF81E03D
:101A5000E8CFEF92FF920F931F93CF937C018B01FE
:101A60000E94AB09C82F811119C08091E80085FD43
:101A70000DC08091E8008E778093E8000E942B0AC9
:101A80000E94AB09882389F3C82F08C0F701819110
:101A90007F018093F1000150110939F78C2FCF910C
:101AA0001F910F91FF90EF9008958091AC020895DF
:101AB00080916602811113C09FB7F8944091A603EC
:101AC0005091A7036091A8037091A9039FBF443C64
:101AD00059406105710518F081E080936602089510
:101AE000EF92FF920F931F93CF93DF93D82F0FB6F0
:101AF00007FE46C08091C002843079F080910601D3
:101B000090E001962091080130E0822393232091F8
:101B100007012817190609F0C9C00E94580D811144
:101B20000FC08091060190E001962091080130E0FD
:101B300082239323209107012817190609F0B6C0C4
:101B40000E947C078C01C091E900CF708091EC006D
:101B500080FD37C080E0C82B83E08093E90085E0FA
:101B6000E82E8091EB0085FD08C08091EB0080FF9E
:101B700004C08091EE0087FD44C0CF70C093E9009F
:101B8000E09106018E2F90E001962091080130E04F
:101B900082239323209107012817190609F47EC098
:101BA0008091040190910501E80FF92FF11DD08378
:101BB000809106018F5F909108018923809306012F
:101BC0006DC080E8C8CFE0910401F0910501E80FF5
:101BD000F11D90818F5F209108018223809307017E
:101BE0009093F1008091E80085FD0BC08091E800A2
:101BF00080FF07C08091E8008E778093E800E09234
:101C000003018091070190910601981741F190918D
:101C1000E80095FDD8CF80E029C01092F1002EC0D9
:101C20008091060190E001962091080130E0822326
:101C30009323209107012817190609F09ECFF090F1
:101C40000301FF2009F499CF0E947C0780179107B8
:101C500009F487CFFA94F09203018C0182CF80912E
:101C6000E80085FFD8CFD093F10081E09091F20099
:101C7000992379F09091E80090FF0BC09091E800D3
:101C800095FDCBCF9091E8009E779093E800E0928D
:101C90000301882329F2CF70C093E90080E0DF912F
:101CA000CF911F910F91FF90EF900895E091060161
:101CB00077CF599A519889B1869581700895893165
:101CC00051F0D8F48D3039F060F4873021F028F4E9
:101CD0008450823020F481E008958930E1F380E07F
:101CE00008958431C1F330F48131A9F38231B9F719
:101CF00082E008958831E0F3F2CF823CC9F358F4D2
:101D00008D3149F318F48A3199F3E9CF8E3181F39B
:101D1000813C29F7E0CF873CF1F228F4843CD9F2EA
:101D2000853C31F3DCCF8A3C18F3D9CFE82FE69518
:101D3000E695E695EF70F0E0E653FD4F9081482F71
:101D4000477021E030E001C0220F4A95EAF787FF93
:101D500004C02095292320830895292BFCCF8330AC
:101D6000C9F128F4813061F0823019F1089585308D
:101D700009F452C008F43FC0863009F45EC00895EB
:101D800080911A01681790F4861B80931A01809144
:101D90001A011F928F938CE49AE09F938F930E9475
:101DA000C4060F900F900F900F90089510921A0193
:101DB000EECF80911901681750F4861B80931901AA
:101DC000809119011F928F938AE39AE0E6CF1092D7
:101DD0001901F6CF80911801681750F4861B809383
:101DE0001801809118011F928F9387E29AE0D5CF56
:101DF00010921801F6CF80911701681750F4861BD6
:101E000080931701809117011F928F9382E19AE0CE
:101E1000C4CF10921701F6CF80911601681750F4C5
:101E2000861B80931601809116011F928F9389EF74
:101E300099E0B3CF10921601F6CF80911501681783
:101E400050F4861B80931501809115011F928F938A
:101E50008EED99E0A2CF10921501F6CF833009F4F0
:101E600045C028F4813061F0823049F10895853011
:101E700009F46AC008F451C0863009F47CC00895A2
:101E800080911A01482F460F5527551F4F3F510586
:101E900094F4680F60931A0180911A011F928F9336
:101EA0008FEC99E09F938F930E94C4060F900F9040
:101EB0000F900F9008958FEF80931A01EDCF8091CE
:101EC0001901482F460F5527551F4F3F510554F410
:101ED000680F60931901809119011F928F938DEB08
:101EE00099E0E0CF8FEF80931901F5CF8091180131
:101EF000482F460F5527551F4F3F510554F4680F83
:101F000060931801809118011F928F938AEA99E0DB
:101F1000C9CF8FEF80931801F5CF80911701482F1B
:101F2000460F5527551F4F3F510554F4680F6093D6
:101F30001701809117011F928F9385E999E0B2CF25
:101F40008FEF80931701F5CF80911601482F460F30
:101F50005527551F4F3F510554F4680F60931601E4
:101F6000809116011F928F938CE799E09BCF8FEFA2
:101F700080931601F5CF80911501482F460F552704
:101F8000551F4F3F510554F4680F60931501809120
:101F900015011F928F9381E699E084CF8FEF809394
:101FA0001501F5CFCF93DF932091C8023091C9027C
:101FB0002817390701F19093C9028093C802E09174
:101FC0009703F09198033097B1F0EC010084F1850C
:101FD000E02D09958091AC038570853061F4DF9325
:101FE000CF938EEF94E09F938F930E94C4060F903F
:101FF0000F900F900F90DF91CF910895CF93DF93C3
:102000002091C6023091C7022817390701F1909339
:10201000C7028093C602E0919703F091980330972E
:10202000B1F0EC010680F781E02D09958091AC03B9
:102030008570853061F4DF93CF9380EF94E09F93B8
:102040008F930E94C4060F900F900F900F90DF9116
:10205000CF910895982F9F779230F1F088F49923CB
:10206000A9F09130B1F01F928F9388EE91E09F9389
:102070008F930E94C4060F900F900F900F9004C092
:10208000933069F09F3779F780E008958078826413
:10209000089580788A6408958078896408958078A6
:1020A00088640895EF92FF920F931F93CF93DF936D
:1020B0008DE791E09F938F930E94C40683E791E0A0
:1020C0009F938F930E94C40688E691E09F938F931D
:1020D0000E94C40607E612E00F900F900F900F9039
:1020E0000F900F90D0E0C0E087E5E82E81E0F82E59
:1020F000F80180818823B1F091811F929F931F92F4
:102100008F9382811F928F93DF93CF93FF92EF92F1
:102110000E94C406EDB7FEB73A960FB6F894FEBF1C
:102120000FBEEDBF21960D5F1F4FC031D10501F7E6
:1021300085E591E09F938F930E94C4060F900F90C6
:10214000DF91CF911F910F91FF90EF90089589EA51
:102150009AE00E942B061F9281E08F931F9285E0E8
:102160008F938BE59AE09F938F930E94C4060F9004
:102170000F900F900F900F900F9008958091AC03E7
:1021800083FF7EC08AE896E00E942B068091A1031F
:102190001F928F9385E896E09F938F930E94C406C9
:1021A00083E896E00E942B068091A203282F082E38
:1021B000000C330B3F938F9380E896E09F938F93AF
:1021C0000E94C4068EE796E00E942B068091A3032E
:1021D000282F082E000C330B3F938F938BE796E04C
:1021E0009F938F930E94C40689E796E00E942B0676
:1021F0008091A403282F082E000C330B3F938F935C
:1022000086E796E09F938F930E94C40684E796E04A
:102210000E942B068091A503282F082E000C330B5B
:102220003F938F9381E796E09F938F930E94C4061C
:102230008EE696E00E942B0680919E031F928F935C
:102240008BE696E09F938F930E94C40689E696E002
:102250000E942B0680919D031F928F9386E696E045
:102260009F938F930E94C40683E696E00E942B06FC
:102270008DB79EB74C960FB6F8949EBF0FBE8DBF1C
:1022800081EA93E00E94F0080E947C079093A003EB
:1022900080939F0308950F931F93CF93DF938091B3
:1022A0009B0390919A03892B8093540290919903F8
:1022B000992389F0892B80935402E5E5F2E02CE51F
:1022C00032E080E0919191118F5F2E173F07D1F797
:1022D000811110929903E0919703F0919803309740
:1022E000B1F10280F381E02D84E592E009958091BF
:1022F000AC0382FF2CC080FF04C088ED95E00E94F3
:102300002B06D0E0C0E002ED15E08091AC0380FF29
:102310000EC0FE01EC5AFD4F80811F928F931F93D8
:102320000F930E94C4060F900F900F900F9021966C
:10233000C830D10551F78091AC0380FF08C080ED13
:1023400095E0DF91CF911F910F910C942B06DF91B7
:10235000CF911F910F91089510929B0310929A03B1
:10236000E4E5F2E011821282138214821582168251
:1023700017820E944B1185E0E1EAF3E0DF011D9234
:102380008A95E9F710929E0310929D030E94BE1059
:1023900090E080E00E94FE0F90E080E00C94D20F6D
:1023A000CF93C82F1F928F9384EA9BE09F938F93C4
:1023B0000E94C40681E090E0A0E0B0E004C0880F75
:1023C000991FAA1FBB1FCA95D2F78093AD039093A4
:1023D000AE03A093AF03B093B0030F900F900F9094
:1023E0000F90CF910C94AC11882341F0809590917F
:1023F0009B03892380939B030C944B11089588239E
:1024000039F090919B03892B80939B030C944B1183
:1024100008958732D8F58E3108F0FCC08E3009F46B
:102420008FC078F4873009F470C08B3009F456C03F
:10243000863009F458C087E697E00E942B0680E0BA
:102440000895863109F4A6C078F48031A1F79091FF
:10245000AC03892F877F93FF88608093AC0383FF51
:102460007FC08DEE98E063C0893109F47CC08B3168
:1024700011F79091AC03892F8D7F91FF826080933B
:10248000AC0381FF5AC086E299E051C0883331F134
:1024900050F4893221F0853311F0873261F680E003
:1024A0000E94D01140C08334D1F320F48A3318F253
:1024B0008953F6CF883409F0BECF0E94AC118CE46A
:1024C00099E00E942B062FEF83ED90E3215080408E
:1024D0009040E1F700C000000E9430098DEA96E0CC
:1024E0000E942B0620C08091AC03817F8E7F809359
:1024F000AC0380E497E00E942B068DE599E00E94F2
:102500002B0681E08093AB0308958091AC0380FF9C
:102510000CC08FE399E00E942B068091AC03817F71
:102520008E7F8093AC0381E0089583E399E00E945D
:102530002B068091AC038160F4CF88E199E0D0CF85
:102540009091AC03892F8B7F92FF84608093AC03C2
:1025500082FF03C089E099E0EACF89EF98E0C0CF1D
:1025600080EE98E0BDCF81ED98E00E942B068EEAC8
:1025700098E00E942B0689E698E00E942B0683E4EF
:1025800098E00E942B068EEF97E00E942B0682EDCA
:1025900097E0A6CF84EC97E00E942B060E940D09DD
:1025A0001F928F938AEA97E09F938F930E94C406AD
:1025B000809114011F928F9383E997E09F938F93EB
:1025C0000E94C4068091AA031F928F9380E897E02F
:1025D0009F938F930E94C4062FB7F8948091A6030F
:1025E0009091A703A091A803B091A9032FBFBF9317
:1025F000AF939F938F9389E697E09F938F930E9469
:10260000C4068DB79EB742960FB6F8949EBF0FBE14
:102610008DBF89CF8D5144CFCF93DF93882309F4A9
:1026200054C09EE7980F933020F5C2E0D9E382387A
:1026300031F0C4E0D7E4833811F4C1E0D3E50E945F
:102640000D098C2309F441C08D2F0E9494070E942C
:102650004B112FEF41EE54E0215040405040E1F744
:1026600000C000008D2F0E948807DF91CF910C944D
:102670004B119CEF980F913AB0F390E2980F98307D
:1026800088F4877021E030E0A90102C0440F551F93
:102690008A95E2F7CA01809590919B0389238093E4
:1026A0009B03E3CF9BE5980F933030F490E080E0FC
:1026B000DF91CF910C94FE0F885A873130F490E06F
:1026C00080E0DF91CF910C94D20FDF91CF910895EC
:1026D000CF93DF93882309F4BDC0C82F8EE78C0FFA
:1026E000833030F5C238F1F0C338F9F0C4E0D7E4F4
:1026F0000E940D098C2309F0ADC08D2F0E94940714
:102700000E944B112FEF81EE94E0215080409040C9
:10271000E1F700C000008D2F0E948807DF91CF9164
:102720000C944B11C2E0D9E3E3CFC1E0D3E5E0CF95
:102730008CEF8C0F813A08F03AC18091AB03813065
:1027400099F040F08230E9F11092AB038C2F0E9497
:102750009407E4CF8091D90287FFF8CF8C2F0E9495
:102760000912811177C0F2CF8091D90287FDF6CF8F
:10277000C431C9F048F4CB3059F0C031C1F08EE01B
:1027800095E00E942B0611C0C93269F0C833B9F731
:1027900080E497E00E942B0684E195E00E942B06DE
:1027A00081E08170DECF1092AB0380E0FACF0E940F
:1027B000A71080E195E00E942B0682E08093AB0396
:1027C000EFCFC432D0F4CE3108F0C0C0CB30E9F046
:1027D00048F4C73009F4D1C08DEB95E0DF91CF917B
:1027E0000C942B06C331C9F1C431B1F78091DA02E0
:1027F000882349F11092DA020AC0CB3409F4BBC035
:10280000C0F4C93299F3C83339F70E94A7108091F8
:10281000DA02882309F4C8C01F928F9387EB95E0F2
:102820009F938F930E94C4060F900F900F900F906C
:1028300011C0C13509F499C0C23509F490C0CE3435
:1028400059F66AE093C08CEC95E00E942B0681E07B
:102850008093AB03DF91CF91089586EA95E00E94C3
:102860002B0684E995E00E942B0680911A011F92A5
:102870008F9381E995E09F938F930E94C4068FE820
:1028800095E00E942B068DE795E00E942B06809133
:1028900019011F928F938AE795E09F938F930E946F
:1028A000C40688E795E00E942B0689E695E00E9421
:1028B0002B06809118011F928F9386E695E09F93D7
:1028C0008F930E94C40684E695E00E942B0683E560
:1028D00095E00E942B06809117011F928F9380E54F
:1028E00095E09F938F930E94C4068EE495E00E942A
:1028F0002B0689E395E00E942B06809116011F921A
:102900008F9386E395E09F938F930E94C40684E3A0
:1029100095E00E942B068DE195E00E942B068091A8
:1029200015011F928F938AE195E09F938F930E94E8
:10293000C40688E195E00E942B068DB79EB74896A5
:102940000FB6F8949EBF0FBE8DBF61CFCE51EC2F56
:10295000F0E0E95BFE4F80818093DA0258CF61E0BE
:102960008091DA020E942E0F52CF61E08091DA024C
:102970000E94AF0E4CCF6AE0F3CF8EE180931A0134
:1029800082E3809319018AE08093180184E18093A7
:10299000170188E08093160188E2809315018FEB80
:1029A00095E00E942B0633CF84EB95E017CF80E2B1
:1029B0008C0F883068F4C77021E030E001C0220F2E
:1029C000CA95EAF780919B03822B80939B03A6CE46
:1029D0008BE58C0F833070F481E890E0C53A31F0DC
:1029E00083E890E0C63A11F482E890E0DF91CF915D
:1029F0000C94FE0F88E58C0F873108F069C082EED9
:102A000090E0C83A09F460C089EE90E0C93A09F450
:102A10005BC08AEE90E0CA3A09F456C085EB90E0BC
:102A2000CB3A09F451C086EB90E0CC3A09F44CC0A3
:102A300083EB90E0CD3A09F447C084EB90E0CE3AC6
:102A400009F442C087EB90E0CF3AF1F18CEC90E0D2
:102A5000C13BD1F18DEC90E0C03BB1F183E891E056
:102A6000C23B91F18AE891E0C33B71F182E991E0C8
:102A7000C43B51F184E991E0C53B31F181E292E040
:102A8000C63B11F183E292E0C73BF1F084E292E0B1
:102A9000C83BD1F085E292E0C93BB1F086E292E01A
:102AA000CA3B91F087E292E0CB3B71F08AE292E080
:102AB000CC3B51F08FE690E0CD3B31F090E080E0F0
:102AC000CE3B11F480E790E0DF91CF910C94D20FD0
:102AD000CF3B09F0BFCE0E94AC119FEF20E782E010
:102AE000915020408040E1F700C000000E94300972
:102AF000CF92DF92EF92FF920F931F93CF93DF93CA
:102B000000D000D01F92CDB7DEB76C0185E0F60192
:102B1000DE01119601900D928A95E1F7F601408150
:102B200051812381348191E02115310531F05F3FDE
:102B300019F491E04F3F09F090E090FD99C0F60143
:102B40000281F580F2949FE0F92249835A830B8336
:102B5000722F3D832C83602F8D810E94AD07182F2B
:102B6000E92FE295EF70EF3008F082C0F0E0E55415
:102B7000FA4E0C94892ACA15CA15081608167E162C
:102B8000B01638163816A21738167818781838166E
:102B900038163419F92FFF70FF2E907F19F0F29438
:102BA00080EFF8220023C9F0FF2039F080919A03CA
:102BB000F82AF0929A030E944B11812F0F900F90E8
:102BC0000F900F900F90DF91CF911F910F91FF9079
:102BD000EF90DF90CF900C946813812F0E940C131C
:102BE000FF2009F445C0F09480919A03F822F092F6
:102BF0009A030F900F900F900F900F90DF91CF914D
:102C00001F910F91FF90EF90DF90CF900C944B119C
:102C1000892F8F70907F903211F08295807F1123E1
:102C200079F0113009F449C0002309F455C0FF20A0
:102C300059F0F601958190FF69C29F70958304C099
:102C4000002321F1F1100FC00F900F900F900F9003
:102C50000F90DF91CF911F910F91FF90EF90DF9038
:102C6000CF900C94FF1121E0F212EECF80939903E4
:102C70000F900F900F900F900F90DF91CF911F91B9
:102C80000F91FF90EF90DF90CF900895F11011C059
:102C9000109299030F900F900F900F900F90DF916B
:102CA000CF911F910F91FF90EF90DF90CF900C94F8
:102CB000F41191E0F912ECCFDBCF002349F0E5E00D
:102CC000EF15B0F290919B03982309F4BDCFE2CFAA
:102CD000F4E0FF1568F2DECFFF20E1F2812F0F90C4
:102CE0000F900F900F900F90DF91CF911F910F9148
:102CF000FF90EF90DF90CF900C940C13892F869566
:102D000086958370C1F0813009F0B2CF812F937026
:102D1000011102C090E080E00F900F900F900F9093
:102D20000F90DF91CF911F910F91FF90EF90DF9067
:102D3000CF900C94D20F812F9370011102C090E0BC
:102D400080E00F900F900F900F900F90DF91CF9138
:102D50001F910F91FF90EF90DF90CF900C94FE0F9A
:102D6000002309F471C0803FA1F40E9408078195F7
:102D70008093A3030F900F900F900F900F90DF910F
:102D8000CF911F910F91FF90EF90DF90CF900C9417
:102D9000BE10813F19F40E940807EACF823F31F448
:102DA0000E94080781958093A203E4CF833F19F422
:102DB0000E940807F8CF893F29F40E94CD0680932E
:102DC000A403D8CF8A3F21F40E94CD068195F7CF86
:102DD0008B3F31F40E94CD0681958093A503CACF25
:102DE0008C3F19F40E94CD06F8CF8091A103816039
:102DF000143FA1F08091A1038260153F79F080918A
:102E0000A1038460163F51F08091A1038860173FB1
:102E100029F0183F31F48091A10380618093A103D0
:102E2000A9CF80919D0381601D3F59F080919D0342
:102E300082601E3F31F01F3F09F09CCF80919D03BF
:102E4000846080939D0396CF803FC1F48091A3035B
:102E500087FD1092A3038091A20381118BCF8091F3
:102E6000A303811187CF8091A403811183CF809127
:102E7000A50381117FCF10929E037CCF813F29F45F
:102E80008091A30318162CF3E6CF8091A203123F82
:102E900029F487FFE0CF1092A203DDCF133F19F48E
:102EA0001816CCF3D8CF193F39F48091A403181623
:102EB00094F61092A403CFCF1A3F29F48091A40373
:102EC00087FFC9CFF6CF1B3F39F48091A50387FF59
:102ED000C2CF1092A503BFCF1C3F29F48091A50358
:102EE0001816BCF3B8CF8091A1038E7F143FA1F0D8
:102EF0008091A1038D7F153F79F08091A1038B7F95
:102F0000163F51F08091A103877F173F29F0183FAA
:102F100031F48091A1038F7E8093A1039CCF809197
:102F20009D038E7F1D3F59F080919D038D7F1E3F35
:102F300031F01F3F09F08FCF80919D038B7F8093ED
:102F40009D0389CF892F837009F064C0011190CE51
:102F5000812F829586958770880F880F412F4F703B
:102F6000C42ED12CF12CE12C082E04C0CC0CDD1C7D
:102F7000EE1CFF1C0A94D2F740E050E0BA0114FFA7
:102F800011C00FE010E020E030E004C0000F111F7E
:102F9000221F331F8A95D2F7B901A8014095509599
:102FA000609570950091AD031091AE032091AF0331
:102FB0003091B0039695969593709230E9F028F58C
:102FC000913089F04C295D296E297F2940235123B6
:102FD000622373234093AD035093AE036093AF031A
:102FE0007093B00345CEC02AD12AE22AF32A4C2995
:102FF0005D296E297F29EECF4C295D296E297F2915
:103000004027512762277327E5CF402351236223AE
:103010007323EDCF8695002311F0892F81708823CB
:1030200009F426CE812F829586958770880F880FA8
:10303000412F4F70C42ED12CF12CE12C082E04C04E
:10304000CC0CDD1CEE1CFF1C0A94D2F740E050E0D3
:10305000BA0114FF11C00FE010E020E030E004C01E
:10306000000F111F221F331F8A95D2F7B901A80143
:10307000409550956095709500911303109114033D
:103080002091150330911603969596959370923082
:10309000E9F028F5913089F04C295D296E297F29C6
:1030A000402351236223732340931303509314034B
:1030B0006093150370931603DBCD0C291D292E296F
:1030C0003F29402B512B622B732BEECF4C295D29CE
:1030D0006E297F294027512762277327E5CF402398
:1030E0005123622373234C295D296E297F29DCCF6C
:1030F000803F09F44EC0D0F480E4810F803270F13B
:10310000002309F4ACC0FF2009F4A6C0812F0E945F
:103110006813193309F099C0FFEF21EE84E0F150F4
:1031200020408040E1F700C00000A2CD823F09F4BA
:1031300070C008F45BC0833F19F7002309F47CC01A
:10314000292F2F7181E090E0A0E0B0E004C0880F4B
:10315000991FAA1FBB1F2A95D2F73AC0E12FE07131
:10316000FE2E892F8F71002351F00E947A08812F43
:103170008295807FF11068CD812F8F7065CD0E9480
:103180005608812F8295807FF11084CD812F8F701A
:1031900081CD002331F1F4E0FF1508F469CD292F2A
:1031A0002F7181E090E0A0E0B0E004C0880F991F8B
:1031B000AA1FBB1F2A95D2F7409113035091140305
:1031C000609115037091160384279527A627B727CA
:1031D0008093130390931403A0931503B0931603E5
:1031E00047CD25E02F1508F443CDD9CF892F8F7116
:1031F000002399F00F900F900F900F900F90DF9198
:10320000CF911F910F91FF90EF90DF90CF900C9492
:103210007A08892F8F71002369F30F900F900F9018
:103220000F900F90DF91CF911F910F91FF90EF9032
:10323000DF90CF900C945608109213031092140351
:10324000109215031092160313CD133509F464CFB1
:10325000173409F00DCD60CF892F8F71CBCFF110CE
:103260003DCD892F8F71D9CF811102CD002309F473
:10327000FFCC0E94AC118FEF90E7E2E081509040CC
:10328000E040E1F700C000000E9430091F93CF9397
:10329000DF938091E002807FB1F48091DD0288238A
:1032A00091F0209112031091E102C091DB02D091C4
:1032B000DC02A091DE02B091DF0241E0CF3F09F0D5
:1032C00040E0121304C0DF91CF911F91089581E077
:1032D000109721F0842FDF3F09F080E030E080FD7F
:1032E00033C0C90166E070E00E94642AFC01EE511F
:1032F000FD4F81818D1328C080818C1325C0828170
:10330000811122C0838194818A1B9B0B883C91058B
:10331000D8F48091E0028F7080618093E002C9014F
:1033200066E070E00E94642AFC01E951FD4F908143
:103330009F70906190838BED92E00E947815DF91F1
:10334000CF911F910C949A082F5F3F4F2770B9CFF0
:103350009F92AF92BF92CF92DF92EF92FF920F9324
:103360001F93CF93DF93CDB7DEB761970FB6F89475
:10337000DEBF0FBECDBF8C0185E0F801DE011D96DA
:1033800001900D928A95E1F7F80140812181F28048
:10339000C380D4809091DB023091DC026091DE0228
:1033A0007091DF0281E06115710531F03F3F19F442
:1033B00081E09F3F09F080E0F82FF1709F2E80FDA3
:1033C0004EC18BEDA82E82E0B82EE090DD02F60112
:1033D000E61BF70BEE2009F404C18091E002582FA0
:1033E000507FE83CF10508F0BDC0511183C0EF2CBF
:1033F000321322C0941320C0F1101EC08F70806160
:103400008093E002C5010E9478158091E002F801E6
:1034100085838E2D61960FB6F894DEBF0FBECDBFAB
:10342000DF91CF911F910F91FF90EF90DF90CF90A0
:10343000BF90AF909F90089581E0C114D10431F006
:103440002F3F19F481E04F3F09F080E080FD14C068
:1034500081E08F25F82FF170BF2EE091120330919B
:10346000E10280FD22C0FF20A1F28091E002816094
:103470008093E002E12CCDCF80E0ECCFF0E0CF01F3
:1034800066E070E00E94642ADC01AE51BD4F1196E7
:103490008C911197281307C08C91481304C0129681
:1034A0008C918F11E0CF3196E770E313E7CF7C2D3D
:1034B000D98AC88A522F6F2D89890E94AD07292F7A
:1034C00022952F70223050F0243078F49F7051F004
:1034D000F8019581907F31F4E92C9BCF9F7011F01A
:1034E0008823D1F3805E8830B8F3C8010E94781534
:1034F0009B2CF2CF321306C0941304C0F801FF20B6
:1035000009F48AC04D872E87FF867C2DD98AC88A08
:10351000522F6F2D89890E94A408882309F4AEC018
:10352000FF2009F4ABC08091E002803270F020915E
:10353000DB023091DC0238872F831986DB86CA864E
:103540008C87CE0107960E94781586E0F801ABEDD6
:10355000B2E001900D928A95E1F70E944619EE249F
:10356000E39457CF51110AC08BED92E00E94781579
:1035700086E0F50111928A95E9F77CCF32130FC0EE
:1035800094130DC0F1100BC0F8018583C8010E948F
:10359000781586E0F50111928A95E9F73ACF4D87C3
:1035A0002E87FF867C2DD98AC88A522F6F2D898954
:1035B0000E94A408882309F461C0FF2009F45EC0BA
:1035C0008091E002803208F22091DB023091DC022F
:1035D0003A8329831B82DD82CC828E83CE010196C1
:1035E000B2CFE83CF105A8F6EF2CFF2009F446C065
:1035F00032131FC094131DC08091E00280FD10C0E3
:10360000982F907F69F0F8018583903F31F0982FD3
:10361000907F905F8F70892B8583C8010E947815F9
:1036200086E0F801ABEDB2E001900D928A95E1F7EA
:10363000F0CE4D872E87FF867C2DD98AC88A522FDF
:103640006F2D89890E94A40881117FCF8091E002AB
:1036500081608093E002C8010E947815DACEFF20D5
:1036600069F04D872E87FF867C2DD98AC88A522F14
:103670006F2D89890E94A408811167CFC8010E941B
:1036800078156DCFCF93DF93CDB7DEB767970FB6C1
:10369000F894DEBF0FBECDBF4B8B5C8B6D8B7E8BEA
:1036A0008F8B1A8A198A85E0FE017396DE011D96BA
:1036B00001900D928A95E1F786E0FE013D96DE01CC
:1036C000179601900D928A95E1F7CE0107960E9418
:1036D000A819811138C086E0FE013796DE011196E7
:1036E00001900D928A95E1F79F8188852A853B8517
:1036F000232B39F08F3F19F481E09F3F19F080E0D0
:1037000001C081E080FD1FC08091E10290E09C013A
:103710002F5F3F4F27703327409112034217130644
:1037200061F166E070E00E94642ADC01AE51BD4F99
:1037300096E0FE01319601900D929A95E1F7209363
:10374000E1020E949A08809112039091E102891788
:1037500009F190E066E070E00E94642A8E519D4F6E
:103760000E94A8198823B1F08091120390E001967D
:103770008770992780931203E6CF0E94AC111092B4
:10378000E1021092120386E0EBEDF2E0DF011D9200
:103790008A95E9F767960FB6F894DEBF0FBECDBFE6
:1037A000DF91CF910895CF93DF9300D01F92CDB7D3
:1037B000DEB72091C002243041F52091130122236D
:1037C00021F123E029839B838A8382E08093E900AF
:1037D0008FEF9091E800815095FD06C095ED9A9588
:1037E000F1F700008111F5CF8091E80085FF0DC051
:1037F00050E040E063E070E0CE0101960E94290DA8
:103800008091E8008E778093E8000F900F900F90E2
:10381000DF91CF910895CF93DF9300D01F92CDB762
:10382000DEB72091C002243081F5209113012223BC
:1038300061F119821A821B8222E029838138910565
:1038400020F0805891099B838A8382E08093E9006D
:103850008FEF9091E800815095FD06C095ED9A9507
:10386000F1F700008111F5CF8091E80085FF0DC0D0
:1038700050E040E063E070E0CE0101960E94290D27
:103880008091E8008E778093E8000F900F900F9062
:10389000DF91CF9108952091C002243049F522E0B4
:1038A0002093E9002FEF3091E800215035FD06C04C
:1038B00035ED3A95F1F700002111F5CF2091E800A0
:1038C00025FF16C02091130150E040E063E070E056
:1038D000222339F021E02093F10050E040E065E040
:1038E00070E00E94290D8091E8008E778093E800B7
:1038F0000895CF93DF932091C002243011F521E089
:103900002093E90021E8215021F03091E80035FFB3
:103910001BC02091E80025FF14C0EC0150E040E0FE
:1039200068E070E00E94290D8091E8008E77809316
:10393000E80088E0FE01ADEAB2E001900D928A95C0
:10394000E1F7DF91CF910895EFE3F1E03197F1F7DF
:1039500000C00000D8CF489906C023E02A95F1F7AF
:1039600000000197C1F70895489B06C023E02A95FF
:10397000F1F700000197C1F70895509A8AEB8A95F4
:10398000F1F700C0509883E091E00197F1F700C093
:1039900000000895509A83E091E00197F1F700C08C
:1039A000000050989AEB9A95F1F700C00895EF92B5
:1039B000FF920F931F93CF93DF93D0E0C0E090E886
:1039C000E92EF12C082F10E0C7010C2E02C09595AE
:1039D00087950A94E2F780239123892B69F00E944E
:1039E000BD1C2196C830D10579F7DF91CF911F9189
:1039F0000F91FF90EF9008950E94CA1CF2CF509A49
:103A000083EF9BE00197F1F700C000000C94BD1C10
:103A1000CF93C82FF8940E94FF1C8C2F8295807F33
:103A200081600E94D71C0E94CA1C8FE193E001971D
:103A3000F1F700C000007894CF910895EF92FF92C3
:103A40001F93CF93DF93182FD62F7A01C22FF894AC
:103A50000E94FF1C812F8295807FD8608D2B0E9451
:103A6000D71C0E94CA1C489927C081E08093650238
:103A700084EF91E00E94AB1C8FE193E00197F1F796
:103A800000C000000E94BD1C10E0D0E0812F012E7C
:103A9000000C990B8C179D0794F00E94CA1C789417
:103AA0008FE193E00197F1F700C00000DF91CF9123
:103AB0001F91FF90EF90089510926502D9CF8E0D5F
:103AC0009F1DFC0180810E94D71C1F5FDFCFCF9319
:103AD000DF9300D0CDB7DEB749832A8322E0AE0161
:103AE0004F5F5F4F0E941E1D0F900F90DF91CF918F
:103AF0000895DF92EF92FF920F931F93CF93DF937E
:103B0000D82FC62F7A01D22E80E0422F50E0282FE6
:103B1000082E000C330B241735070CF1F8940E9483
:103B2000FF1C8D2F8295807FCC608C2B0E94D71C30
:103B30000E94CA1C489919C081E08093650284EFF5
:103B400091E00E94AB1C892B99F488EE93E09F933F
:103B50008F930E94C40678940F900F9010C02E0D82
:103B60003F1DF90110828F5FD2CF10926502E7CF1F
:103B700084EF91E00E94B41C892B51F4789480E08A
:103B8000DF91CF911F910F91FF90EF90DF900895FB
:103B900088E290E00E94AB1C892B19F486EE93E03A
:103BA000D6CF84E690E00E94B41CC0E0892B21F4BB
:103BB00084EE93E0CCCFC82F82E890E00E94AB1C4B
:103BC000DC2FD695D695D6958823E9F08C01112760
:103BD000C8010E94B41C8823B1F0DD1578F4F70108
:103BE000ED0FF11D9081990F22E830E0201B310B81
:103BF000081B11092017310794F0908381E08C0F86
:103C0000CF3FC9F6C0E078948FE193E00197F1F7D8
:103C100000C000008C2F869586958695B1CF916067
:103C2000ECCFCF93DF93CDB7DEB728970FB6F894DC
:103C3000DEBF0FBECDBF28E0AE014F5F5F4F0E94D9
:103C4000791D823071F489819A8198278927982774
:103C500028960FB6F894DEBF0FBECDBFDF91CF918F
:103C6000089590E080E0F4CFCF93DF93D82FC62F54
:103C700062E00E94111EEFE3F6E03197F1F700C019
:103C80000000887F2C2F2770282B492F62E08D2F72
:103C9000DF91CF910C94671D1F93CF93DF93182F63
:103CA00060E00E94111EEC0180E0209701F1DF939B
:103CB000CF931F921F9389EF91E09F938F930E9460
:103CC000C4068D2F99270F900F900F900F900F9093
:103CD0000F908F3F910529F00E942A1081110E94B8
:103CE000960ECE0199278F3F910529F481E0DF914F
:103CF000CF911F9108958C2F0E942A108823B1F331
:103D00000E94960EF3CF0F931F93CF93DF9385E915
:103D100091E09F938F930E94C4060F900F90C1E093
:103D2000D0E008E811E063E08C2F0E94111E00979C
:103D300071F09F938F93DF93CF931F930F930E9404
:103D4000C4060F900F900F900F900F900F90219638
:103D5000C031D10541F786E891E09F938F930E948F
:103D6000C4060F900F90DF91CF911F910F9108958E
:103D7000FF920F931F93CF93DF93F82E00910001D2
:103D8000109101018FEF9FEF90930101809300014B
:103D90000F3F100769F560E08F2D0E94111E8C0106
:103DA000009749F11F938F938F2D90E063E070E0AF
:103DB0000E94642A89599D4FFC0181811F928F9333
:103DC0001F92FF928DE991E09F938F930E94C4060A
:103DD0008DB79EB708960FB6F8949EBF0FBE8DBFE5
:103DE0000F37100779F48FE70E94960E81E004C028
:103DF0000115110541F580E0DF91CF911F910F91E1
:103E0000FF9008950F3F100709F58FEF0E94960E5F
:103E10000E94831E0E945210E9CF8A3089F5C07833
:103E2000C2632EC0823061F18C2F0E94960EDF3F5C
:103E3000E9F28D2F90E0982F88278F6F90930101E2
:103E400080930001D3CF0F37100769F2C12FD02F15
:103E50001F3F11F4C02FDFEF8F2D90E063E070E083
:103E60000E94642A89599D4FFC0181810E945F0E46
:103E70008130C1F68C2F8F77823379F6C078CA6093
:103E80008C2F8F778A3281F6C078C067CDCFAF9202
:103E9000BF92CF92DF92EF92FF920F931F93CF9337
:103EA000DF9300D000D01F92CDB7DEB7D82E90E0C0
:103EB00063E070E00E94642A89599D4FFC010281F1
:103EC00025E0CE0101967C01AC0160E08D2D0E94C1
:103ED000791D182F80E0123008F40AC11F920F9349
:103EE0001F92DF928AED91E09F938F930E94C40608
:103EF0000F900F900F900F900F900F90670184ED2F
:103F0000A82E81E0B82EF60181916F011F928F9348
:103F1000BF92AF920E94C4068C2D8E190F900F9005
:103F20000F900F90811778F381ED91E09F938F931D
:103F30000E94C4060F900F900C3441F5898191E0E6
:103F4000582F507486FF90E02A81422F40743B81A5
:103F500032FF18C08F77898330FF16C02F772A83EE
:103F600088E031FF88E88B83552319F08B818067C7
:103F70008B8380E0442321F08B8187608B8381E0F9
:103F800013E01CC08068E7CF2068E9CF0D3409F04A
:103F9000C3C09B818A81292F87FFBAC020682B83E9
:103FA00097FFB8C080688A83FE01E10FF11D808110
:103FB00086FB992790F982FB882780F948EF58E81B
:103FC000153009F065C19D81492F50E080E093FFD5
:103FD00080E897FF80649C81E92FF0E093FF806286
:103FE00097FF80619B81A92FB0E093FF886097FFC6
:103FF00084609A8197FF8260298127FF8160809386
:10400000C102BD0133E0660F771F3A95E1F7607892
:1040100073708F0136E0000F111F3A95E1F700270A
:104020001C71602B712B2F77622B9A01322F222764
:10403000330F2227307E622B732B9F779A01322F0A
:1040400022273295330F307E292BB695BA2FAA2717
:10405000B795A795A078B3702A2B3B2BFE2FEE27A0
:10406000FF0FFF0FEE27FC712E2B3F2BA9012138EC
:10407000FFEF3F0714F441E85FEF4038510514F0BB
:104080004FE750E0FB0161389FEF790714F4E1E856
:10409000FFEFE038F10514F0EFE7F0E010925C027A
:1040A00010925D0210925E0210925F021092C402A2
:1040B0004093C202E093C3021F921F927F936F93BB
:1040C000FF93EF933F932F935F934F931F928F93A1
:1040D0008EEA91E09F938F930E94C40681EC92E058
:1040E0000E94F0080FB6F894DEBF0FBECDBF81E08E
:1040F0000F900F900F900F900F90DF91CF911F9125
:104100000F91FF90EF90DF90CF90BF90AF90089508
:104110002F7745CF8F7747CF023409F044C079819C
:104120006A8166FB882780F976FB992790F914301D
:1041300009F4ACC091E0F72FF07476FF90E081E0D5
:10414000E62FE07466FF80E02B8130E0A901B5E046
:10415000440F551FBA95E1F7D90114E0AA0FBB1F10
:104160001A95E1F74A2340787F77472B4983A901C5
:1041700006E0440F551F0A95E1F740786F77642BEE
:104180006A83A9015695542F44275795479530E7E0
:10419000F11101C030E0342B2FE0E11101C028E023
:1041A000322B3B83EDCE0F3221F00F3511F0063666
:1041B00081F5498191E0F42FF07446FF90E06A8127
:1041C00081E0E62FE07466FF80E07B81272F30E0FE
:1041D00070FB47F94983A901A6E0440F551FAA9532
:1041E000E1F740786F77462B4A83B5E0220F331F03
:1041F000BA95E1F720787870272B30E7F11101C0EC
:1042000030E0232B37E0E11101C030E0232B2B837A
:10421000B7CE033059F5498191E0E42FE07446FFB1
:1042200090E06A8181E0762F707466FF80E02B81D8
:1042300030E020FB47F94983A901F5E0440F551F01
:10424000FA95E1F740786F77462B4A83A6E0220F74
:10425000331FAA95E1F7207830E7E11101C030E083
:10426000232B3FE07111D2CF38E0D0CF043009F4D6
:104270009BCE023309F498CE998196FB992790F949
:104280002A8126FB882780F920682A8312E096CEAF
:10429000212F012E000C330BF701E20FF31F9111B8
:1042A0000BC05083882331F0F701E20FF31F208108
:1042B000276020831F5F84CE4083F4CF2F923F92EC
:1042C0004F925F926F927F928F929F92AF92BF9226
:1042D000CF92DF92EF92FF920F931F93CF93DF93D2
:1042E000CDB7DEB760970FB6F894DEBF0FBECDBF77
:1042F0001091020120916302309164024FB7F8944B
:104300008091A6039091A703A091A803B091A9035F
:104310004FBF821B930B0B9748F5209160023091A1
:1043200061024FB7F8948091A6039091A703A091E2
:10433000A803B091A9034FBF821B930B883E934003
:1043400008F4CFC10E947C079093610280936002C1
:10435000AA24A394B12C10E040901B0150901C01A2
:1043600060901D0170901E018A2C65C10E947C071F
:10437000909364028093630200E07E0189E0E80E7E
:10438000F11C36EDA32E33E0B32E40ED842E43E036
:10439000942E5DEC652E53E0752E1F7009F453C00A
:1043A000C12ED12CC60163E070E00E94642A8959B5
:1043B0009D4FFC0180818230D1F188F5882309F47A
:1043C00062C028E0A70160E0812F0E94791D582E6D
:1043D0008823A9F1C60163E070E00E94642A89592C
:1043E0009D4FFC0182811F928F93DF92CF92BF92EB
:1043F000AF920E94C4060F900F900F900F900F90F5
:104400000F9067018C2D8E19851508F448C07F9296
:104410006F920E94C4060F900F9001E010C083308D
:1044200051F0873071F6812F0E944C1E07C0812FFA
:104430000E94B81E03C0812F0E94471F082F809141
:104440006502882329F01F5F809102018113A5CFA7
:104450001F70109302018091620281112EC00E9490
:10446000590E811106C08FE70E94960E81E080935D
:104470006202002309F451CF0E947C0790936102ED
:10448000809360022EC1133031F0173031F01230BA
:10449000D1F682E0CDCF83E0CFCF87E0C5CFF60164
:1044A00081916F011F928F939F928F920E94C406F9
:1044B0000F900F900F900F90A5CF0E94590E882358
:1044C000C1F28FEF0E94960E10926202D2CFDF925D
:1044D0008F93BF92AF9287EB93E09F938F930E944D
:1044E000C406E7E6F2E00F900F900F900F900F9048
:1044F0000F900FE010E0F02EE02E912E85A588237E
:1045000009F499C20150110933970730110599F741
:104510002F923F9280EA93E0A2C2C80163E070E06C
:104520000E94642A89599D4FFC018082C80163E082
:1045300070E00E94642A89599D4FFC012183C801C3
:1045400063E070E00E94642A89599D4FFC01228338
:104550003F932F931F930F932F923F9280E793E007
:104560009F938F930E94C4060FB6F894DEBF0FBED0
:10457000CDBF92E08912D8C063E0802F0E94111E47
:104580006C01009769F41F930F938DE292E09F9363
:104590008F930E94C4060F900F900F900F904AC007
:1045A000DF928F931F930F9387E192E09F938F93F6
:1045B0000E94C4068C2D0E945F0E0F900F900F90EA
:1045C0000F900F900F90882309F4A5C0813009F453
:1045D000A5C0823009F0A5C080E391E09F938F933E
:1045E0009F92EF9285E092E09F938F930E94C40682
:1045F00023E04D2D63E08F2D0E94671D63E08F2D1A
:104600000E94111E282F8E2D992D63E070E00E94CC
:10461000642A89599D4FFC0122830E940D09682F4D
:1046200060958F2D0E94341E0F900F900F900F9069
:104630000F900F9011E063E0882D0E94111E6C0115
:104640003A2C2B2C009709F042CFC50163E070E0B3
:104650000E94642A89599D4FFC018081882361F062
:10466000C50163E070E00E94642A89599D4FFC01F6
:1046700010821182128211E02FEFA21AB20A88E092
:10468000A816B10409F070CE87E6C82E82E0D82EB5
:1046900098E0E92EF12C00E063E08E2D0E94111EBF
:1046A000892B81F4F601808D882361F0C70163E0D6
:1046B00070E00E94642A89599D4FFC01108211828A
:1046C000128201E0FFEFEF1AFF0A23E0C20ED11CB5
:1046D00080E1E816F10401F7111101C001110E94F7
:1046E000521080E060960FB6F894DEBF0FBECDBFCB
:1046F000DF91CF911F910F91FF90EF90DF90CF90BE
:10470000BF90AF909F908F907F906F905F904F90F1
:104710003F902F90089587E291E060CF8CE291E086
:104720005DCF84E391E05ACFF3E08F1273C163E071
:10473000802F0E94111E6C01009729F41F930F9384
:1047400082E493E024CFDF928F931F930F938CE248
:1047500093E09F938F930E94C4061C2D0F900F909F
:104760000F900F900F900F901F3231F01F3521F0F6
:10477000163611F0123461F449825A826B827C82BF
:1047800024E0AE014F5F5F4F61E08F2D0E941E1D40
:104790008FEF810F823008F052C024E04D2D63E08E
:1047A0008F2D0E94671D63E08F2D0E94111E6C01EA
:1047B000F4E08F1709F446C023E04D2D63E08F2D00
:1047C0000E94671D63E08F2D0E94111E6C01182F3F
:1047D000833089F427E040E062E08F2D0E94671D5E
:1047E0008E2D992D63E070E00E94642A89599D4FB7
:1047F000FC0112831FCF8130D9F422E04D2D63E0FC
:104800008F2D0E94671D63E08F2D0E94111E6C0189
:10481000182F813069F49F92EF9285E193E09F9386
:104820008F930E94C4060F900F900F900F90D8CFD7
:10483000123029F49F92EF928EEF92E0F0CF143075
:1048400009F082C028E0AE014F5F5F4F61E08F2D1D
:104850000E94791D863008F44DC02D813E8132279B
:104860002327322798851F928F931F929F933F9300
:104870002F931F929F938F811F928F938E811F92F0
:104880008F938D811F928F938C811F928F938B8139
:104890001F928F938A811F928F9389811F928F938A
:1048A0009F92EF9283EB92E09F938F930E94C406B6
:1048B0000FB6F894DEBF0FBECDBF89818B3409F0EF
:1048C00063C08A818D34D9F48B818C3409F09BC00C
:1048D0008C81813309F097C09F92EF92EDE9F2E06D
:1048E000FF93EF930E94C4060F900F900F900F90CC
:1048F00014E076CF882309F324E630E0B3CF8F3479
:1049000009F081C08B81893409F07DC08C818435A8
:1049100009F079C08F2D0E94081D22E44D2D63E01F
:104920008F2D0E94671D63E08F2D0E94111E182F8E
:104930009F92EF9289E892E09F938F930E94C40622
:104940000F900F900F900F90123309F049CF9F9264
:10495000EF928EE392E09F938F930E94C40688E0CB
:10496000EFE1F1E0DE01119601900D928A95E1F7F9
:104970008F2D0E94081D28E0AE014F5F5F4F62E05F
:104980008F2D0E941E1D4FCF8A3951F58A8180528A
:104990008230C8F59F92EF9289E792E09F938F93C0
:1049A0000E94C40621E840E061E08F2D0E94671D4F
:1049B00021E841E061E08F2D0E94671D21E842E07F
:1049C00061E08F2D0E94671D28E343E061E08F2D99
:1049D0000E94671D0F900F900F900F901CE400CF66
:1049E0008C3489F48A81843571F49F92EF9280E649
:1049F00092E09F938F930E94C4060F900F900F90A8
:104A00000F901DE4EDCE9F92EF9280E592E09F9390
:104A10008F9368CFF7E08F120DCE1F930F9383E52E
:104A200093E09F938F930E94C40611E00F900F9024
:104A30000F900F9000CE4D2D407F402B2EEF63E066
:104A4000882D0E94671D63E0802F0E94111E9C012B
:104A5000892B09F062CD2F923F928CE893E09F93CF
:104A60008F930E94C4060F900F900F900F9003CE6B
:104A700078941F920F920FB60F9211248F939F93E9
:104A8000AF93BF938091A6039091A703A091A80331
:104A9000B091A9030196A11DB11D8093A603909327
:104AA000A703A093A803B093A903BF91AF919F91CF
:104AB0008F910F900FBE0F901F9018951F920F921D
:104AC0000FB60F9211248F939F93AF93BF93809152
:104AD0009C03811113C08091A6039091A703A0911C
:104AE000A803B091A9034196A11DB11D8093A6030F
:104AF0009093A703A093A803B093A903BF91AF918C
:104B00009F918F910F900FBE0F901F9018951F923D
:104B10000F920FB60F9211242F933F934F935F93F1
:104B20006F937F938F939F93AF93BF93EF93FF9375
:104B30008091E10082FF09C08091E20082FF05C000
:104B40008091E1008B7F8093E1008091E10080FF04
:104B50001FC08091E20080FF1BC08091E2008E7F29
:104B60008093E2008091E20080618093E200809176
:104B7000D80080628093D80019BC85E08093C00281
:104B80008091AC028093AB021092AC020E94AC11F7
:104B90008091E10084FF2DC08091E20084FF29C054
:104BA00084E089BD86E089BD09B400FEFDCF809117
:104BB000D8008F7D8093D8008091E1008F7E809314
:104BC000E1008091E2008F7E8093E2008091E2001C
:104BD00081608093E2008091B702882309F440C08D
:104BE00084E08093C0020E94AC118091AB0280935C
:104BF000AC028091E10083FF22C08091E20083FF3C
:104C00001EC08091E100877F8093E10082E0809365
:104C1000C0021092B7028091E1008E7F8093E10084
:104C20008091E2008E7F8093E2008091E2008061BB
:104C30008093E20042E060E080E00E94F909FF9189
:104C4000EF91BF91AF919F918F917F916F915F9104
:104C50004F913F912F910F900FBE0F901F9018957D
:104C60008091E30087FD02C081E0BBCF83E0B9CF34
:104C7000CF93DF93CDB7DEB72C970FB6F894DEBF96
:104C80000FBECDBF84B7877F84BF0FB6F894A895B9
:104C900080916000886180936000109260000FBE78
:104CA00080E890E00FB6F8948093610090936100E3
:104CB0000FBE80E79DE0909353018093520189E0FD
:104CC00091E090939803809397038DE294E00E9483
:104CD0002B060E941909809163008E7F80936300E8
:104CE00081E08093AA021092E2001092E10080918C
:104CF000D8008F778093D8008091D8008068809307
:104D0000D8008091D8008F7D8093D80084E089BD41
:104D100086E089BD09B400FEFDCF1092C00210925A
:104D2000B7021092B6021092B50242E060E080E055
:104D30000E94F9098091E1008E7F8093E1008091CB
:104D4000E20081608093E2008091E20088608093BD
:104D5000E2008091E0008E7F8093E000789482E012
:104D600084BD93E095BD9AEF97BD80936E008091CE
:104D7000C002843009F070C10E94580D882309F4E4
:104D80006BC18BE194E00E942B068091AC038160A3
:104D90008093AC0387E992E0E7E6F2E010821182AB
:104DA000128233968E179F07C9F78AED92E0BAEC0C
:104DB000CB2EB2E0DB2EF60111926F018E179F070A
:104DC000D1F7569A5E9A58985098599A5198509A95
:104DD0008FED9EE20197F1F700C0000050980E940D
:104DE000831E569A5E988DE094E00E942B06F2E0B6
:104DF0004F2EF4E05F2EA8E16A2E712C8091C00244
:104E0000853009F42CC10E945E2108E912E0EAEC29
:104E1000AE2EE2E0BE2E312CF50121905F01F801AB
:104E20009080921409F468C08091AC0381FF40C067
:104E300085EF93E00E942B062AEC32E03C872B871B
:104E4000F12CE12CEB85FC852191FC87EB872295E9
:104E500030E0C901880F991F880F991F8C7C359508
:104E60002795359527952373822B90E027E331E032
:104E70003F932F939C01220F331F2A7A9595879594
:104E80008575822B1F928F93FF92EF928AEE93E0AB
:104E90009F938F930E94C406FFEFEF1AFF0A0FB68D
:104EA000F894DEBF0FBECDBF30E1E316F10451F63A
:104EB000E12CFF24F3949224892D8F21C1F0EE82FE
:104EC0003F8291E08F2D822109F490E098870E9423
:104ED0007C078160782F9A8789874E815F816885FA
:104EE0008A850E94421BF80180818F258083E3948C
:104EF000FF0CF8E0EF12E0CF33940F5F1F4F20E17B
:104F000032128ACF3FEF39833A831B820E947C079B
:104F10008160782F9D838C8349815A816B818D813B
:104F20000E94421B80919F039091A0032FB7F89499
:104F30004091A6035091A7036091A8037091A90323
:104F40002FBFFA01E81BF90B20919E0380911901F4
:104F500090E0211107C080911A0190E06AE070E0B2
:104F60000E94642AE817F90780F08091A203F0906C
:104F7000A3031091A4030091A5038111A6C0F11011
:104F800066C1111164C1011162C10E940D099091A5
:104F90009702891761F10E940D0980939702909101
:104FA000AC039570953051F41F928F935F924F929E
:104FB0000E94C4060F900F900F900F90F0909702F0
:104FC00007E612E08FE0E82EF094F80185A5823024
:104FD00021F46F2D8E2D0E94341EEA940350110986
:104FE000F7E0EF12F2CF6F2D82E00E94341E209185
:104FF000E4003091E5008091A8029091A902281761
:10500000390739F18091E4009091E5009093A9026D
:105010008093A8020E94580D8823D9F08091C00285
:105020008430B9F48091E9008F709091EC0090FF8A
:10503000BAC090E8892B93E09093E9009091EB003F
:1050400090FF04C09091EE0097FDCBC08F708093CD
:10505000E9000E942B0AD2CE0E942B0A88CE8091B2
:10506000C002843011F110929C0380E40FB6F894D2
:10507000A895609260000FBE8093600083B7817F27
:10508000846083BF83B7816083BF7894889583B73A
:105090008E7F83BF0FB6F894A895809160008861D9
:1050A00080936000109260000FBE8091B60288234A
:1050B00009F4A4CE0E945E21EAECF2E08191811114
:1050C000B0C0CE16DF06D1F799CE2F3F19F02F5F73
:1050D00020939E03181624F40E9408078093A203CD
:1050E0008091A20387FF05C00E94080781958093E5
:1050F000A2031F1424F40E9408078093A303809145
:10510000A30387FF05C00E94080781958093A3032E
:105110006091A203662331F1F090A303FF2011F107
:10512000062E000C770B880B990B0E94632923E352
:1051300033E343E35FE30E94C7290E942B29609376
:10514000A2036F2DFF0C770B880B990B0E9463292C
:1051500023E333E343E35FE30E94C7290E942B2943
:105160006093A303111624F40E94CD068093A40338
:105170008091A40387FF05C00E94CD06819580938E
:10518000A403101624F40E94CD068093A5038091F9
:10519000A50387FF05C00E94CD0681958093A503D6
:1051A0000E94BE10F2CE90E045CFE0910401F09154
:1051B0000501E90FF11D20819F5F309108019323C4
:1051C000909307012093F1009091E80095FD09C0AC
:1051D0009091E80090FF05C09091E8009E77909331
:1051E000E8009091070120910601291721F02091F4
:1051F000E80025FDDACF9091F200992309F426CF3B
:105200009091E80090FF22CF9091E80095FD06C0B4
:105210009091E8009E779093E80018CF1092F100EB
:10522000F3CF84E089BD86E089BD09B400FEFDCFDF
:105230008091D8008F7D8093D8008091E0008260BB
:105240008093E0008091E00081FDFCCFD7CD2F3F1F
:1052500009F03DCF4ECF0E9432296894B1110C94D1
:10526000C12908950E94A62988F09F5798F0B92F68
:105270009927B751B0F0E1F0660F771F881F991F8B
:105280001AF0BA95C9F714C0B13091F00E94C02944
:10529000B1E008950C94C029672F782F8827B85F54
:1052A00039F0B93FCCF3869577956795B395D9F7E3
:1052B0003EF490958095709561957F4F8F4F9F4FED
:1052C0000895E89409C097FB3EF4909580957095F9
:1052D00061957F4F8F4F9F4F9923A9F0F92F96E942
:1052E000BB279395F695879577956795B795F111B7
:1052F000F8CFFAF4BB0F11F460FF1BC06F5F7F4F54
:105300008F4F9F4F16C0882311F096E911C0772365
:1053100021F09EE8872F762F05C0662371F096E86E
:10532000862F70E060E02AF09A95660F771F881F3D
:10533000DAF7880F9695879597F9089557FD905855
:10534000440F551F59F05F3F71F04795880F97FB49
:10535000991F61F09F3F79F0879508951216130603
:105360001406551FF2CF4695F1DF08C01616170632
:105370001806991FF1CF8695710561050894089567
:10538000E894BB2766277727CB0197F908950E94F9
:10539000D9290C94532A0E94452A38F00E944C2A9D
:1053A00020F0952311F00C943C2A0C94422A0C9482
:1053B000C1290E949E2978F39923C9F35523B9F393
:1053C000950F50E0551FAA27EE27FF27BB27002483
:1053D0000894679520F4E20FF31FB41F0A1E220FF2
:1053E000331F441FAA1F6695A9F7779530F4F30F72
:1053F000B41F0A1E121E08F46395330F441FAA1F20
:10540000221F769599F7879520F4B40F0A1E121E75
:10541000631F440FAA1F221F331F8695A9F7862FEB
:10542000712D602D11249F5750409AF0F1F0882380
:105430004AF0EE0FFF1FBB1F661F771F881F91509A
:105440005040A9F79E3F510580F00C943C2A0C94E3
:10545000C1295F3FE4F3983ED4F38695779567952D
:10546000B795F795E7959F5FC1F7FE2B880F911DC4
:105470009695879597F9089597F99F6780E870E06A
:1054800060E008959FEF80EC089500240A941616BA
:10549000170618060906089500240A941216130622
:1054A000140605060895092E0394000C11F48823B0
:1054B00052F0BB0F40F4BF2B11F460FF04C06F5FCC
:1054C0007F4F8F4F9F4F08950024552704C0080E2B
:1054D000591F880F991F009729F076956795B8F3A3
:1054E0007105B9F7802D952F089597FB072E16F4B7
:1054F000009407D077FD09D00E948F2A07FC05D0C1
:105500003EF4909581959F4F0895709561957F4FDA
:105510000895EE0FFF1F0590F491E02D0994AA1B4A
:10552000BB1B51E107C0AA1FBB1FA617B70710F08E
:10553000A61BB70B881F991F5A95A9F780959095C0
:0A554000BC01CD010895F894FFCFDF
:10554A00FFFF030554010000FF550D791C4B1C0B8E
:10555A001CD31B01012808140A321E00001007B5CB
:10556A0014000069FFFF37414E53490049534F0069
:10557A004A4953003F3F3F00407F2215019600747D
:10558A0000580471048A0401020304050607080985
:02559A0000000F
:106800008800EA44E944E244040005000600070069
:10681000080009000A000B000C000D000E000F001C
:1068200010001100120013001400150016001700CC
:10683000180019001A001B001C001D001E001F007C
:10684000200021002200230024002500260027002C
:10685000280029002A002B002C002D002E002F00DC
:10686000300031A132003300340035A1360037004A
:10687000380082003A003B003C003D003E003F00F3
:1068800040004100420043004400450046004700EC
:10689000480049004A004B004C004D004E004F009C
:1068A00050005100520053002E0054005500560075
:1068B000580059005A005B005C005D005E005F00FC
:1068C0006000610062006300640000005700850002
:1068D000CD440000000000000000000000000000A7
:1068E000000000000000A520890087008A008B00BE
:1068F000E000E100E200E300E400E500E600000063
:106900000100010001000100EA4401000100E2442D
:106910000100010001000100460001004A004B0097
:10692000010001004700480001000100E9440100A6
:106930000100010001000100010001003A003B00DC
:106940003C003D003E003F0040004100420043004B
:10695000010035004C0001000100440045005200D8
:1069600049000100010050004F0029004D004E0079
:1069700051000100010001000100010001000100BF
:1069800001000100010001000100010001000100FF
:1069900001000100010001000100010001004D00A3
:1069A0004A004E004B0001000100010001000100FF
:1069B00001000100010001000100010001000100CF
:1069C00001000100010001000100000001000100C0
:1069D00001000000000000000000000000000000B6
:1069E000000000000000010049000100010001005A
:1069F0000100010001000100010001000100000090
:00000001FF
